S020000062696E2F64656D6F70726F675F656B5F6C6D3373363936352E7372656358
S11380006C080020158200002986000029860000E3
S113801029860000298600002986000029860000A0
S11380202986000029860000298600002986000090
S11380302986000029860000298600001986000090
S11380402986000029860000298600002986000070
S11380502986000029860000298600002986000060
S11380602986000029860000298600002986000050
S11380702986000029860000298600002986000040
S11380802986000029860000298600002986000030
S11380902986000029860000298600002986000020
S11380A02986000029860000298600002986000010
S11380B02986000029860000298600002986000000
S11380C029860000298600002986000029860000F0
S11380D029860000298600002986000029860000E0
S11380E029860000298600002986000029860000D0
S11380F0EE11AA5510B50120C1F2000049F26D2419
S1138100C0F20004A0470120C2F20000A0474FF0D3
S11381104020032149F21903C0F20003984749F2B1
S11381208D43C0F20003984701464FF44040C4F227
S113813000004FF46142602349F64504C0F2000494
S1138140A04710BD10B540F24503C2F200031B78EE
S1138150EBB94FF44040C4F2000049F68913C0F271
S113816000039847B0F1FF3F4BD040F20003C2F246
S11381700003187040F24503C2F2000301221A7092
S113818040F24403C2F2000300221A7010BD40F210
S11381904403C2F200031B785C1C4FF44040C4F259
S11381A0000049F68913C0F200039847B0F1FF3F7D
S11381B027D040F20003C2F20003185540F24402F3
S11381C0C2F2000211780131C9B211701B788B42DE
S11381D017D140F24503C2F2000300221A7040F2A4
S11381E00003C2F200035B78FF2B0AD140F20003C4
S11381F0C2F200039B7823B949F2B523C0F200030D
S1138200984710BD08B549F2B523C0F2000398475A
S113821008BD00BF10B517498D4640F20002C2F2F6
S1138220000240F20003C2F200039A4210D2131D6E
S11382300F4CE41A24F003040434002310464BF2D8
S1138240B811C0F200015A581A500433A342FAD1AB
S113825009480A494FF000028842B8BF40F8042B8D
S1138260FADB48F25D53C0F20003984710BD00BF2B
S1138270030000206C080020000000206C07002090
S113828010B52020C2F2000049F26D23C0F20003B1
S113829098474FF4A044C4F202042046012148F652
S11382A0CD73C0F20003984720460121002248F60E
S11382B09D73C0F20003984710BD00BF10B548F28B
S11382C00D63C0F200039847044640F24803C2F22B
S11382D000031B68C31AB3F5FA7F2BD340F24C0397
S11382E0C2F200031B7883B940F24C03C2F20003CC
S11382F001221A704FF4A040C4F20200114648F65D
S11383009D73C0F2000398470FE040F24C03C2F2A1
S1138310000300221A704FF4A040C4F202000121AD
S113832048F69D73C0F20003984740F24803C2F236
S113833000031C6010BD00BF10B548F22D63C0F2ED
S11383400003984748F20D64C0F20004A04740F2CD
S11383505403C2F2000300F5FA701860A04740F21B
S11383605003C2F2000300F51C501030186049F6A7
S11383704933C0F20003984740F22413C2F20003C9
S11383804FF6A9621A8043F61371598040F2201304
S1138390C2F200034FF6FF7119800021598040F2A8
S11383A01C13C2F200031A8040F213125A804EF6D4
S11383B0030049F67D33C0F20003984748F2516345
S11383C0C0F20003984710BD08B540F2EC03C2F2B6
S11383D000031B7813F0400F11D113F0020F0ED0DD
S11383E040F2F003C2F200031B681A79FF2A06D197
S11383F05B7923B948F20523C0F20003984708BD0E
S113840010B548F2D973C0F200039847002853D03E
S113841040F2E002C2F20002108040F22813C2F2DD
S113842000039C894FF400604AF67533C0F20003E0
S1138430984784421CD1012049F6B133C0F20003AD
S1138440984740F2E003C2F200031B88A3B34AF644
S11384503163C0F20003984748F62D03C0F20003CD
S1138460984740F2E003C2F2000300221A8023E09E
S113847040F22813C2F200039C8940F606004AF633
S11384807533C0F200039847844215D14AF6F1438C
S1138490C0F20003984740F2E003C2F200031B88D5
S11384A053B148F62D03C0F20003984740F2E003AD
S11384B0C2F2000300221A8048F20D63C0F20003E6
S11384C0984740F25403C2F200031B6898422BD32E
S11384D040F25402C2F2000203F5FA73136040F250
S11384E0F403C2F2000340F2F802C2F200021A607E
S11384F0022049F6B133C0F20003984740F2E0038A
S1138500C2F200031B887BB14AF63163C0F2000358
S1138510984748F62D03C0F20003984740F2E00361
S1138520C2F2000300221A8048F20D63C0F2000375
S1138530984740F25003C2F200031B6898420CD3E0
S113854040F25002C2F2000203F51C5310331360D0
S11385504AF69943C0F20003984710BD08B54FF49A
S11385606070C0F2C01049F2D123C0F200039847F2
S113857048F28123C0F20003984748F2C553C0F281
S11385800003984748F23933C0F20003984748F291
S1138590F503C0F20003984748F2BD26C0F2000676
S11385A048F20145C0F2000548F24514C0F2000447
S11385B0B047A847A047FBE740F25803C2F20003C4
S11385C01960FEE708B549F28D43C0F200039847ED
S11385D044F6D353C1F26203A3FB0020800949F29D
S11385E07173C0F20003984749F24973C0F2000363
S11385F0984749F25D73C0F20003984740F25C0368
S1138600C2F2000300221A6008BD00BF40F25C03FE
S1138610C2F200031868704740F25C03C2F2000320
S11386201A6801321A607047FEE700BF10B54FF4B4
S1138630A044C2F21004204649F26D23C0F20003A4
S11386409847204649F20523C0F20003984710BD1D
S11386502DE9F04385B02020C2F2000049F26D23D9
S1138660C0F2000398474FF4A040C4F202000C216A
S113867049F26503C0F2000398474FF40044C4F282
S1138680040420467F2148F6D533C0F200039847FE
S11386902046002148F62543C0F2000398470146CE
S11386A0204648F65943C0F20003984749F28D43E7
S11386B0C0F2000398470146204648F67513C0F2FD
S11386C0000398472046162148F6B113C0F2000370
S11386D09847204648F69923C0F20003984720465D
S11386E0012148F6A143C0F200039847044648F22A
S11386F00D63C0F20003984700F59C5708374FF408
S11387000048C4F204084FF0010948F6A146C0F23B
S1138710000648F20D65C0F2000506E040464946F1
S1138720B0470446A847874202D914F0040FF5D095
S113873008238DF8083000238DF8093027238DF89D
S11387400A3069238DF80B305B238DF80C304523F8
S11387508DF80D3001A8694648F6ED43C0F20003D8
S11387609847019BB3F1FF3F13D0009AB2F1FF3F4A
S11387700FD08DF80830190A8DF809101B0C8DF8EC
S11387800A308DF80B20130A8DF80C30120C8DF87A
S11387900D204FF40040C4F2040002A948F621233E
S11387A0C0F20003984740F26C03C2F200039DF844
S11387B008201A709DF809205A709DF80A209A70B2
S11387C09DF80B20DA709DF80C201A719DF80D208D
S11387D05A7105B0BDE8F08338B54FF40044C4F2D3
S11387E004042046002148F62543C0F200039847BC
S11387F005462046294648F65943C0F200039847E7
S113880015F0010F0FD04FF40040C4F2040040F201
S11388102811C2F2000140F2426248F6E123C0F29C
S11388200003984738BD002038BD00BF08B540F2AA
S1138830E003C2F200034FF40040C4F2040040F22B
S11388402811C2F200011A8848F65D33C0F2000311
S1138850984708BD2DE9F001844600F1100403692E
S11388601FFA83F8180C08701B0E4B70A8F1060051
S11388709042B4BF074617463E1F012E06DD022371
S11388802568CD500433B342FADD00E002239F4251
S11388901DDDDCF81050FE1E9E4209D18D55394471
S11388A02B0A01F8023C2D0C01F8015C7B1C0EE044
S11388B0BE1E9E4206D18D5539442D0A01F8015C35
S11388C0BB1C04E07E1E9E4204BF8D55FB1CA8F118
S11388D002018B4203DA256804338B42FBDB9042AE
S11388E0C8BF4042BDE8F001704700BF70B440F219
S11388F0FE739A42C8BF504239DCA2F10E030C78D1
S113890043EA04434C7843EA046300F1100603612C
S1138910151F012D06DD0223CC5834600433AB420D
S1138920FADD00E0022393421ED0D41E9C420BD1F8
S11389300C5D114411F8025C11F8013C1B0443EA7C
S11389400523234303610FE0941E9C4207D10B5D72
S1138950114411F8011C43EA0123036104E0541E8D
S11389609C4204BF0B5D036101238363104670BC0A
S1138970704700BF38B504460D464FF40042C4F2B8
S11389800402904209D04BF2A800C0F200004E212C
S113899048F2B952C0F2000290474CF66B23C6F677
S11389A05F33A3FB0523C3F34753636238BD00BFA2
S11389B038B504460D464FF40043C4F2040398420C
S11389C009D04BF2A800C0F20000952148F2B95337
S11389D0C0F20003984725F4873333F0160209D018
S11389E04BF2A800C0F20000992148F2B953C0F23A
S11389F000039847E36823F01603EAB21343E360E5
S1138A00A36823F00E03C5F307221343A360E36BAB
S1138A1023F00103C5F307451D43E56338BD00BFDB
S1138A2030B583B005460C464FF40043C4F204034A
S1138A3098420AD04BF2A800C0F200004FF48171B2
S1138A4048F2B953C0F20003984754B94BF2A80056
S1138A50C0F2000040F2031148F2B953C0F200031F
S1138A60984723788DF8043063788DF80530A3781F
S1138A708DF80630E3788DF80730019B6B61002395
S1138A80019323798DF8043063798DF80530019BC7
S1138A90AB6103B030BD00BF10B504464FF40043D2
S1138AA0C4F2040398420AD04BF2A800C0F20000BA
S1138AB04FF4AC7148F2B953C0F200039847A3686D
S1138AC043F01003A360A36843F00103A360E368C9
S1138AD043F00103E360A36843F01003A36010BDF7
S1138AE070B504460E4615464FF40043C4F2040321
S1138AF098420AD04BF2A800C0F2000040F27F2155
S1138B0048F2B953C0F20003984756B94BF2A80093
S1138B10C0F200004FF4207148F2B953C0F20003D0
S1138B209847002D0ADC4BF2A800C0F2000040F286
S1138B30812148F2B953C0F200039847636B13F0E4
S1138B403F0F08D0204631462A4648F65503C0F266
S1138B500003984770BD002070BD00BF70B5044687
S1138B600E4615464FF40043C4F2040398420AD05B
S1138B704BF2A800C0F2000040F28E3148F2B95323
S1138B80C0F20003984756B94BF2A800C0F20000A7
S1138B9040F28F3148F2B953C0F200039847002DD8
S1138BA00ADC4BF2A800C0F200004FF4647148F2F2
S1138BB0B953C0F200039847A36B13F0010FFBD124
S1138BC0204631462A4648F6ED03C0F20003984792
S1138BD070BD00BF38B504460D464FF40043C4F2DF
S1138BE0040398420AD04BF2A800C0F2000040F2FD
S1138BF0354148F2B953C0F20003984735F07F037A
S1138C000AD04BF2A800C0F200004FF4876148F28A
S1138C10B953C0F200039847636823EA0505656009
S1138C2038BD00BF38B504460D464FF40043C4F2C6
S1138C30040398420AD04BF2A800C0F200004FF49B
S1138C408B6148F2B953C0F20003984720680DB114
S1138C506368184038BD00BF38B504460D464FF46C
S1138C600043C4F2040398420AD04BF2A800C0F2B5
S1138C70000040F28D4148F2B953C0F20003984716
S1138C8035F07F030AD04BF2A800C0F200004FF485
S1138C90926148F2B953C0F200039847256038BD89
S1138CA038B504460D464FF40043C4F20403984219
S1138CB00AD04BF2A800C0F2000040F2DC4148F2B6
S1138CC0B953C0F20003984704F12003226A12F05A
S1138CD0010FF9D1ED00EDB245F001051D601A68F0
S1138CE012F0010FFBD1206B80B238BD38B50C46B1
S1138CF0054650B94BF2C400C0F2000040F26B21AB
S1138D0048F2B953C0F20003984754B94BF2C40077
S1138D10C0F200004FF41B7148F2B953C0F20003D3
S1138D2098474FF46043C4F20F031B6813F0E04FFD
S1138D3019D04FF46043C4F20F031A680023C7F23A
S1138D40FF031340B3F1805F10D04EF2E013C4F27E
S1138D500F031B682B604EF2E413C4F20F031B686D
S1138D602360002038BD4FF0FF3038BD4FF0FF3096
S1138D7038BD00BF20F480534FF40042C4F2050212
S1138D80934218BFB3F1402F31D04FF4C041C4F225
S1138D9000014FF42042C4F20502934218BF8B42F3
S1138DA027D04FF48041C4F202014FF44042C4F290
S1138DB00502934218BF8B421DD04FF4C041C4F248
S1138DC002014FF46042C4F20502934218BF8B4281
S1138DD013D04FF45042C4F203020023C4F206033A
S1138DE0984218BF904214BF002001207047012010
S1138DF0704701207047012070470120704700BF71
S1138E0070B504460E46154648F67553C0F2000385
S1138E10984748B94BF2DC00C0F20000E42148F264
S1138E20B953C0F200039847022D09D94BF2DC0074
S1138E30C0F20000E62148F2B953C0F2000398479B
S1138E4015F0010F04F58063D4F8002414BF3243F5
S1138E50B2431A6015F0020F04F58463D4F8202499
S1138E6014BF164322EA06061E6070BDF8B5044618
S1138E700D4617461E4648F67553C0F20003984740
S1138E8050B94BF2DC00C0F200004FF4DD7148F23F
S1138E90B953C0F20003984727F008027B1E042A46
S1138EA018BF012B0AD94BF2DC00C0F200004FF4CA
S1138EB0DF7148F2B953C0F200039847A6F10803E2
S1138EC0052B0BD956B14BF2DC00C0F2000040F286
S1138ED0C51148F2B953C0F20003984717F0010FC7
S1138EE004F5A063D4F8002514BF2A43AA431A60EA
S1138EF017F0020F04F20453D4F8042514BF2A43D4
S1138F00AA431A6017F0040F04F5A163D4F80825E6
S1138F1014BF2A43AA431A6017F0080F04F5A36389
S1138F20D4F8182514BF2A43AA431A6016F0010F77
S1138F3004F20C53D4F80C2514BF2A43AA431A6034
S1138F4016F0020F04F5A263D4F8102514BF2A43C7
S1138F50AA431A6016F0040F04F21453D4F814252B
S1138F6014BF2A43AA431A6016F0080F04F21C53D4
S1138F70D4F81C2514BF2A43AA431A602EB904F559
S1138F80A563D4F82825154305E004F5A563D4F8B2
S1138F90282522EA05051D60F8BD00BF70B504460A
S1138FA00D46164648F67553C0F20003984750B96B
S1138FB04BF2DC00C0F200004FF4517148F2B95397
S1138FC0C0F20003984744F8256070BD38B50546E3
S1138FD00C4648F67553C0F20003984750B94BF25B
S1138FE0DC00C0F2000040F2044148F2B953C0F280
S1138FF00003984728462146012248F60163C0F23F
S113900000039847284621460122082348F66D6448
S1139010C0F20004A04738BD38B505460C4648F6F2
S11390207553C0F20003984750B94BF2DC00C0F20C
S1139030000040F21F5148F2B953C0F200039847B0
S113904028462146022248F60163C0F200039847ED
S1139050284621460122082348F66D64C0F2000424
S1139060A04738BD38B505460C4648F67553C0F2DE
S11390700003984750B94BF2DC00C0F2000040F204
S1139080C65148F2B953C0F2000398472846214616
S1139090022248F60163C0F200039847284621469D
S11390A00422082348F66D64C0F20004A04738BDCA
S11390B030B420F08053A3F58012013A4FF480714C
S11390C0C0F210018B4218BF012A98BF012040F260
S11390D097804FF40071C0F210014FF48062C0F227
S11390E01002934218BF8B4208BF012000F0888011
S11390F04FF4A041C2F2100100F16042013A8842EB
S113910018BF012A98BF01207AD90422C2F20002B2
S1139110904208BF012073D01022C2F20002904294
S113912008BF01206CD02022C2F20002904208BF86
S1139130012065D020F480148021C2F200014FF494
S11391408072C2F20002944218BF8B4208BF012011
S113915056D020F00052B0F1102F18BF402A08BF9B
S113916001204DD04FF48041C1F200018C4208BF70
S1139170012045D0B0F1101F08BF012040D04FF4AA
S11391808075C1F200054FF40071C1F200018842FC
S113919018BFA84208BF012032D01025C1F2000533
S11391A02021C1F200018A4218BFAA4208BF01204F
S11391B026D00821C1F2100188421CD000F1704170
S11391C00139012917D90421C1F200018C4214D0BC
S11391D0B0F1202F13D00121C2F2100188420ED029
S11391E04FF48050C0F21000834218BF082A14BF05
S11391F00020012004E0012002E0012000E0012021
S113920030BC704710B582B0044649F2B103C0F2D5
S11392100003984750B94BF25010C0F2000040F2DE
S1139220B91148F2B953C0F2000398474BF27413D2
S1139230C0F20003220F53F822201368A1B2C4F332
S1139240044401FA04F42343136000230193019BB3
S11392500F2B05D8019B01330193019B0F2BF9D9E7
S1139260136823EA0404146002B010BD10B5044668
S113927049F2B103C0F20003984750B94BF25010C1
S1139280C0F200004FF4FC7148F2B953C0F200037D
S113929098474BF26813C0F20003220F53F82230B0
S11392A01A68A1B2C4F3044401FA04F414431C6020
S11392B010BD00BF4EF60C53CEF200030422C0F2E0
S11392C0FA521A60FEE700BF01387FF4FDAF704721
S11392D070B504464FF46043C4F20F031B6813F0E7
S11392E0E04F0BD04FF46043C4F20F031A6800231D
S11392F0C7F2FF031340B3F1805F02D1002CC0F228
S1139300C3804EF26002C4F20F0211684EF2700381
S1139310C4F20F031E6821F4800545F4006546F489
S113932000601560186011F0020F02D014F0020FF3
S113933005D011F0010F24D014F0010F21D164F0F5
S113934003031D404EF26003C4F20F031D600028A6
S113935004DA06F03003302B04D00BE005F03003C0
S1139360302B07D14FF4805049F2C923C0F20003D7
S1139370984706E04FF4002049F2C923C0F20003E5
S1139380984725F45F5525F0300543F2F0732340E8
S11393901D434DF68F73C7F6FF73334043F40062E9
S11393A042F23003C8F200032340134304F00802DE
S11393B04EF25801C4F20F014020086053EAC2067D
S11393C00AD54EF27003C4F20F031E604EF260031E
S11393D0C4F20F031D6009E04EF26003C4F20F03F0
S11393E01D604EF27003C4F20F031E60102049F298
S11393F0C922C0F20002904725F0F86020F0030073
S11394000323C0F2C0732340184326F0FC5604F033
S1139410FC510E4314F0804F1FBF40F4800026F42B
S113942080050023C4F240031ABF23401D4326F0E5
S1139430804514F4006F17D14EF25003C4F20F03A9
S11394401B6813F0400F0BD147F6FF734EF2500127
S1139450C4F20F010A6812F0400F01D1013BF9D1A7
S113946020F4006025F400654EF26003C4F20F039B
S113947018604EF27003C4F20F031D60102049F20D
S1139480C923C0F20003984770BD00BF30B44EF248
S11394906003C4F20F0319684EF27003C4F20F03A1
S11394A01A68002AB4BF02F0700301F03003202BC5
S11394B071D003D87BB1102B16D037E1602B00F0AC
S11394C0C180702B00F0BB80302B08BF03F5EA434A
S11394D000F0CF802AE14BF2F403C0F20003C1F3A1
S11394E0841053F82030C4E04FF46043C4F20F03F7
S11394F01B6813F0E04F04BF4EF2C013C0F2E40344
S113950000F0B7804FF46043C4F20F0318680023DF
S1139510C7F2FF030340B3F1805F00F096804FF47D
S11395206043C4F20F0318680023C7F2FF0303402B
S11395300020C1F20100834208D14FF46043C4F219
S11395400F031B689BB2022B00F084804FF460432E
S1139550C4F20F0318680023C7F2FF03034000207E
S1139560C1F2030083421CBF4FF41053C0F2F40352
S11395707FD14FF46043C4F20F031C68A4B24FF4CC
S1139580D853C0F2B7034FF41050C0F2F400002CCB
S113959018BF03466DE04FF46043C4F20F031B6829
S11395A013F0E04F04BF43F67003C0F2390360D0F8
S11395B04FF46043C4F20F0318680023C7F2FF039B
S11395C00340B3F1805F4AD04FF46043C4F20F0309
S11395D018680023C7F2FF0303400020C1F2010012
S11395E0834207D14FF46043C4F20F031B689BB25C
S11395F0022B39D04FF46043C4F20F0318680023E0
S1139600C7F2FF0303400020C1F2030083421CBFE2
S11396104FF41063C0F23D032BD14FF46043C4F206
S11396200F031C68A4B24CF2C063C0F22D034FF4C4
S11396301060C0F23D00002C18BF034619E04FF43F
S1139640004316E04FF4800313E04EF2C013C0F25F
S1139650E4030EE04FF4D853C0F2B70309E043F635
S11396607003C0F2390304E04CF2C063C0F22D036E
S1139670FFE7002A03DA12F4006F03D058E011F474
S1139680006F5AD14EF26400C4F20F0000684FF428
S11396906044C4F20F04246814F0E04F0BD04FF47C
S11396A06044C4F20F0425680024C7F2FF042C4070
S11396B0B4F1805F0AD1C0F34814023404FB03F30D
S11396C000F01F040234B3FBF4F309E0C0F34814C0
S11396D004FB03F300F01F0401346400B3FBF4F350
S11396E010F4804F18BF5B0810F4004F18BF9B089C
S11396F0002AA8BF41F4800112DA12F0804F09D089
S113970012F4006F06D15B00C2F386520132B3FB40
S1139710F2F016E0C2F3C5500130B3FBF0F010E0F4
S1139720C1F3C3500130B3FBF0F00AE0002008E0BD
S113973011F4800FE1D1184603E011F4800FEFD14A
S1139740184630BC704700BF4EF21003CEF200033F
S11397501A6842F005021A60704700BF4EF2100307
S1139760CEF200031A6842F002021A60704700BF8A
S113977010B5441EB4F1807F09D34BF28010C0F2BF
S11397800000D02148F2B953C0F2000398474EF2CA
S11397901403CEF200031C6010BD00BF20F48052FD
S11397A04FF44043C4F200039A4208D04FF460439C
S11397B0C4F20003984214BF002001207047012026
S11397C0704700BF10B5044649F29D73C0F2000310
S11397D0984750B94BF29810C0F200004FF4CF7183
S11397E048F2B953C0F200039847E36A43F0100308
S11397F0E362236B43F4407343F00103236310BD1E
S113980010B5044649F29D73C0F20003984750B95D
S11398104BF29810C0F200004FF4DF7148F2B953D4
S1139820C0F200039847A36913F0080FFBD1E36A61
S113983023F01003E362236B23F4407323F001034A
S1139840236310BDF8B504460E4615461F4649F27B
S11398509D72C0F20002904750B94BF29810C0F2CA
S1139860000040F20D1148F2B953C0F200039847CA
S113987055B94BF29810C0F200004FF4877148F2CA
S1139880B953C0F2000398474FF46042C4F20F0288
S1139890136813F0E04F08BF102340D04FF4604327
S11398A0C4F20F031A680023C7F2FF031340B3F195
S11398B0805F08BF102332D04FF46043C4F20F031B
S11398C01A680023C7F2FF0313400022C1F2010209
S11398D0934209D14FF46043C4F20F031B689BB257
S11398E0022B08BF10231AD04FF46043C4F20F03B5
S11398F01A680023C7F2FF0313400022C1F20302D7
S1139900934218BF08230AD14FF46043C4F20F03F3
S11399101B689BB2002B0CBF10230823FFE705FB39
S113992003F3B3420AD94BF29810C0F2000040F29C
S11399300F1148F2B953C0F200039847204649F684
S11399400102C0F200029047B6EB051F236B3DBF36
S113995043F0200323636D0823F0200328BF23630F
S1139960F600B6FBF5F50135EB096362C5F3450571
S1139970A562E7620023A361204649F2C573C0F2E1
S113998000039847F8BD00BF10B5044649F29D7323
S1139990C0F20003984750B94BF29810C0F200008F
S11399A040F2094148F2B953C0F200039847A36951
S11399B013F0100F0CBF20684FF0FF3010BD00BF34
S11399C030B4013A8D18A94214D20B461C785A7847
S11399D002EB042292B2104480B2824284BF01306E
S11399E080B202339D42F1D8CB432B4423F00103D0
S11399F002331944A94207D10B781B02184480B2E0
S1139A00834284BF013080B230BC704770B540F2ED
S1139A102814C2F20004667C143E237C06EB032661
S1139A20B6B2304480B204F11A01082249F6C115D5
S1139A30C0F20005A84704F122013246A8470346B4
S1139A4020B1000A40EA032080B270BD4FF6FF70D7
S1139A5070BD00BF70B4C4780C44E4B240F2E803B3
S1139A60C2F20003DC700D0A82782A44D2B29A70E2
S1139A7046785E700078187095420DD90136F6B2BA
S1139A8040F2E803C2F200035E702EB940F2E8032C
S1139A90C2F2000301301870C9B28C4217DA0132E5
S1139AA0D2B240F2E803C2F200039A707AB940F2EB
S1139AB0E803C2F200035A780132D2B25A7032B9C2
S1139AC040F2E803C2F200031A7801321A7070BC43
S1139AD0704700BF10B5014640F2F404C2F200041E
S1139AE02068083049F65523C0F2000398472268DD
S1139AF040F2E803C2F200031978117259785172E6
S1139B0099789172DB78D37210BD00BF08B500203C
S1139B100849142249F6C113C0F2000398470346CA
S1139B2020B1000A40EA032080B208BD4FF6FF705E
S1139B3008BD00BF3601002008B5062049F60D23F4
S1139B40C0F20003984708BD40F21813C2F20003A4
S1139B5000221A8040F2F803C2F200035A7640F25F
S1139B607403C2F2000301221A7040F26803C2F2C5
S1139B7000034FF480621A80704700BF40F2740300
S1139B80C2F2000300221A7040F21813C2F200035A
S1139B901B882BB940F21813C2F2000318807047D7
S1139BA040F27403C2F2000301221A70704700BF2E
S1139BB038B540F2F403C2F200031C6840F2F0032B
S1139BC0C2F20003AD4A1A6040F2E403C2F2000399
S1139BD01A60032816D1637E03F00F03032B40F0B1
S1139BE0AE87238A002B40F0AA8740F2EC03C2F22E
S1139BF0000308221A7048F2C933C0F200039847E0
S1139C0000F0CCBD022840F0A78040F26403C2F209
S1139C100003DA780132D2B2DA70C2B940F26403D6
S1139C20C2F200039A780132D2B29A707AB940F241
S1139C306403C2F200035A780132D2B25A7032B9C4
S1139C4040F26403C2F200031A7801321A7040F23F
S1139C50E003C2F2000300221A8040F26A73C2F2E7
S1139C6000031A80637E03F0FD02052A09D1A37E56
S1139C700133DBB2A376782B04BF0023637600F0B4
S1139C805EBF002B00F05B87228A002A52D0A27E9E
S1139C90511EA176002A40F05287E27E082A05D0A0
S1139CA0591EC9B2012917D8052A15D10023637694
S1139CB040F2EC03C2F2000380221A7048F2C93366
S1139CC0C0F20003984740F22813C2F200031422A2
S1139CD083F82F2000F0AABE042A9DBF03219140DF
S1139CE0C9B23021A1760132E27603F00F03013BC1
S1139CF0072B00F22487DFE813F06D020800100040
S1139D00D8042207D8042207D80440F22813C2F248
S1139D100003002283F82F2063E240F2EC03C2F236
S1139D20000304221A7048F2C933C0F200039847B2
S1139D3000F085BD03F00F03032B40F0008740F2D1
S1139D40EC03C2F2000308221A7048F2C933C0F2CD
S1139D500003984700F022BD40F22813C2F200032A
S1139D609B7B452B40F0EB8640F22813C2F20003A4
S1139D70197C5A7C02EB012040F2E003C2F200039A
S1139D801B88984200F3DB8684B240F2E003C2F2FF
S1139D9000031C8040F22813C2F200031B7D13F061
S1139DA03F0F40F0CC8640F22813C2F200035B7DE3
S1139DB0002B40F0C48640F22413C2F200031D8835
S1139DC02DB940F22413C2F200035B88A3B140F220
S1139DD02813C2F20003DB8BAB4240F0B08640F2A2
S1139DE02812C2F2000240F22413C2F20003128CC1
S1139DF05B889A4240F0A38649F60D33C0F2000313
S1139E0098474FF6FF73984240F0998640F2281322
S1139E10C2F20003DB7D062B32D0012B40F08F868B
S1139E2040F22813C2F2000393F82230082B40F0CA
S1139E30868640F22813C2F20003002283F822200F
S1139E409A8C4FF6F6739A4240F22813C2F200033A
S1139E508CBF093208329A8440F22813C2F20003FC
S1139E605A8BDA839A8B1A845D8340F22412C2F2ED
S1139E70000252889A8300F05BBE00BF5E0100209E
S1139E8049F63933C0F2000398474FF6FF739842FE
S1139E9040F0558640F2F803C2F20003597E81B3C4
S1139EA040F22812C2F2000240F2F803C2F20003A8
S1139EB0928C9B889A4224D140F22812C2F200026A
S1139EC040F2F803C2F20003528CDB889A4218D1A4
S1139ED040F22812C2F2000240F2F803C2F2000378
S1139EE0528B1B889A420CD140F22812C2F2000213
S1139EF040F2F803C2F20003928B5B889A4200F0AE
S1139F00918140F22813C2F2000393F82F3003F03A
S1139F103F03022B1CD140F22813C2F200039A8C97
S1139F2040F26003C2F200031A8040F27403C2F2EA
S1139F3000030021197040F21813C2F200031B88B9
S1139F4093427BD040F27403C2F2000301221A70E0
S1139F5040F22813C2F2000393F82F3013F0040FD9
S1139F6040F0ED8540F22813C2F20003142283F876
S1139F702F2040F2E002C2F2000228211180502278
S1139F8083F82E2093F8295093F82D2083F8292064
S1139F9093F8284093F82C2083F8282083F82C4049
S1139FA093F8270093F82B2083F8272083F82B00BD
S1139FB093F8262040F27401C2F200010A7093F86B
S1139FC02A1083F8261083F82A20691CC9B283F862
S1139FD02D10C1B9611CC9B240F22813C2F20003AA
S1139FE083F82C1079B9411CC9B240F22813C2F28B
S1139FF0000383F82B1031B940F22813C2F2000396
S113A000013283F82A2040F22813C2F20003598C4B
S113A01040F26002C2F2000211809A8C5A84998440
S113A0205A8BDA839A8B1A8440F22412C2F2000209
S113A0301188598352889A8300F047BD40F2F8038F
S113A040C2F200035B7E23B1072B40F08C8500F045
S113A05082BD40F2F401C2F2000140F2F803C2F200
S113A06000030B6003219976197600219975042069
S113A070D875D9769A8040F22814C2F20004628C12
S113A080DA80628B1A80A28B5A800120587640F2C3
S113A0906402C2F2000211781973517859739178ED
S113A0A09973D278DA73188294F82920DA7294F8C2
S113A0B028209A7294F827205A7294F826201A724B
S113A0C049F6D523C0F20003984794F82E3003F0E4
S113A0D0F002502A7ADD1B095C1FA40040F27503CC
S113A0E0C2F200031A78002340F22811C2F20001E0
S113A0F05AE0CA1892F8362072B940F27401C2F2DA
S113A10000010B7040F27503C2F200031A7040F2B2
S113A110F804C2F200045DE0012A02D10133DBB28B
S113A12042E0022A2BD10D1895F83750042D26D180
S113A13040F27402C2F20002137040F27503C2F2DC
S113A140000302221A7040F22813C2F200030344EF
S113A15093F8382093F8393043EA022240F260033E
S113A160C2F200031A8040F20A639A4238BF1346CF
S113A17040F2F804C2F200046382A3822AE0084495
S113A18090F8370070B940F27401C2F200010B700C
S113A19040F27503C2F200031A7040F2F804C2F2EE
S113A1A0000417E00344DBB21846A342A1DB40F2EB
S113A1B07401C2F200010B7040F27503C2F2000395
S113A1C01A7040F2F804C2F2000403E040F2F8040A
S113A1D0C2F2000440F22813C2F20003102283F8F2
S113A1E02F2040F22813C2F2000393F82F2042F0EC
S113A1F0020283F82F20022283F83620042283F8F7
S113A2003720062283F838200A2283F8392040F2C6
S113A210E002C2F200022C211180602283F82E2079
S113A22000F011BC40F2F403C2F2000340F2F80261
S113A230C2F200021A6040F2EC03C2F200030022F0
S113A2401A7040F22813C2F2000393F82F3013F06F
S113A250040F11D040F2F803C2F200035A7640F220
S113A260EC03C2F2000320221A7048F2C933C0F290
S113A2700003984700F063BC40F22812C2F20002C7
S113A28092F82E000009800040F27402C2F200022B
S113A2901070143C201A80B240F2E002C2F20002B4
S113A2A0108001F00F01022903D103F03F02122AAA
S113A2B01DD010B913F0030F19D040F22811C2F2C7
S113A2C0000140F2F802C2F20002C98C12899142E4
S113A2D040F0A18340F22811C2F2000140F2F802DA
S113A2E0C2F20002098D5289914240F0948313F026
S113A2F0100F7AD040F2F803C2F20003198A002941
S113A30073D003F10C0049F65523C0F200039847BB
S113A31040F22813C2F2000393F82A4040F2E80303
S113A320C2F200031B78A3425FD140F22813C2F2A9
S113A330000393F82B0040F2E803C2F200035B78B9
S113A340834252D140F22813C2F2000393F82C1036
S113A35040F2E803C2F200039B788B4245D140F2FD
S113A3602813C2F2000393F82D2040F2E803C2F24E
S113A3700003DB78934238D140F2F803C2F20003C1
S113A3801C7358739973DA73DB7E03BB40F2F803D2
S113A390C2F20003987D197E9A7E891AA1EBD0013E
S113A3A0C9B2CAB20844C0B2987512F0800F1CBF7B
S113A3B04A42D2B240F2F803C2F20003D97DA1EBC3
S113A3C091010A44D2B2DA7502EBD0021A7640F255
S113A3D0EC03C2F2000301221A7040F2F803C2F245
S113A3E000031A7E9A7600221A8240F2F803C2F21F
S113A3F000035A7E02F00F03013B072B00F29F83F8
S113A400DFE813F00800400013016F02C202F702F4
S113A4100903540240F2EC03C2F200031B7813F068
S113A420010F00F08C8340F2F803C2F20003032210
S113A4305A7640F2EC02C2F200024021117000226E
S113A4401A8240F2E003C2F20003188850B140F2CD
S113A450EC03C2F2000342221A7049F6D523C0F27B
S113A4600003984740F26A73C2F2000300221A8084
S113A47048F2C933C0F20003984740F2F804C2F22C
S113A48000048BE140F2EC03C2F200031B7813F0EA
S113A490010F00F0B78040F22813C2F2000393F8D2
S113A4A02F3003F03F03122B40F0AC8040F228130E
S113A4B0C2F2000393F82E3003F0F002502A6DDD4F
S113A4C01B095C1FA40040F27503C2F200031A7852
S113A4D0002340F22811C2F2000152E0CA1892F897
S113A4E0362052B940F27401C2F200010B7040F2FE
S113A4F07503C2F200031A7050E0012A02D101333D
S113A500DBB23EE0022A2BD10D1895F83750042D0A
S113A51026D140F27402C2F20002137040F27503B5
S113A520C2F2000302221A7040F22813C2F200039E
S113A530034493F8382093F8393043EA022240F276
S113A5406003C2F200031A8040F20A639A4228BFF1
S113A5501A4640F2F803C2F200035A829A821DE0BE
S113A560084490F8370050B940F27401C2F2000177
S113A5700B7040F27503C2F200031A700EE003443C
S113A580DBB21846A342A9DB40F27401C2F2000117
S113A5900B7040F27503C2F200031A7040F2F80423
S113A5A0C2F200040323637640F22813C2F20003CC
S113A5B093F82620227293F82720627293F82820B9
S113A5C0A27293F82930E372012049F6D523C0F230
S113A5D00003984740F2EC03C2F2000342221A70CF
S113A5E00022228240F2E003C2F200031A8040F209
S113A5F06A73C2F200031A8048F2C933C0F200033E
S113A6009847CBE040F2EC03C2F2000320221A7018
S113A61048F2C933C0F20003984740F2F403C2F28F
S113A62000031B6800225A7692E440F22813C2F217
S113A630000393F82F3013F0010F3ED012F0100FE7
S113A6403BD140F2F803C2F200031B8A002B40F016
S113A650768240F2E004C2F200042088013080B225
S113A66049F6D523C0F20003984740F2EC03C2F246
S113A67000031A7842F010011970238833B140F2B4
S113A680EC03C2F2000342F012021A7048F2C9331A
S113A690C0F20003984740F2F804C2F20004012318
S113A6A02382082363760023E37640F22813C2F260
S113A6B00003112283F82F20B8E113F0200F18D0E3
S113A6C040F22813C2F2000393F83400000293F816
S113A6D0351040F2F003C2F2000340EA01051C68A1
S113A6E02C441C6040F2E003C2F200031888411BB2
S113A6F0198040F2E003C2F20003188878B112F026
S113A700100F0CD140F2EC03C2F200031A7842F0AD
S113A71002021A7049F6D523C0F20003984740F2AA
S113A7202813C2F2000393F8302093F8313003EB7E
S113A73002239BB240F26002C2F20002138040F294
S113A740F802C2F20002928A934200D823B940F27E
S113A7506003C2F200031A8040F2F803C2F200035D
S113A76040F26002C2F2000212885A8240F2EC0304
S113A770C2F200031B7813F0030F00F0E08140F2F3
S113A7806A73C2F2000300221A8048F2C933C0F28D
S113A7900003984740F2F804C2F2000440F2EC03CC
S113A7A0C2F200031B7813F0200F0ED040F26A733C
S113A7B0C2F2000300221A80627640F22813C2F229
S113A7C00003142283F82F2030E113F0100F12D06D
S113A7D040F26A73C2F2000300221A80012323822A
S113A7E004236376E27640F22813C2F200031122B6
S113A7F083F82F201AE140F26A72C2F20002128832
S113A800DAB113F0010F1CBF0023238201D1218A86
S113A81071B9618A8A4282BF40F26A73C2F200034C
S113A820198040F26A73C2F200031B88238204E099
S113A83040F26A73C2F2000319800023E37640F207
S113A840F003C2F2000340F2E402C2F20002126812
S113A8501A6040F26A73C2F200031B887BB1238A38
S113A8606BB140F2E002C2F200022833138040F2DE
S113A8702813C2F20003182283F82F20DCE040F2F0
S113A880EC03C2F200031B7813F0020F00F05781AF
S113A89040F2E003C2F2000328221A8040F2281397
S113A8A0C2F20003102283F82F20C5E040F2EC032B
S113A8B0C2F200031B7813F0010F00F0408140F254
S113A8C0F803C2F2000300225A7640F2EC03C2F20B
S113A8D0000310221A7048F2C933C0F200039847EB
S113A8E02DE140F2E003C2F20003188820B149F6DA
S113A8F0D523C0F20003984740F22813C2F20003A4
S113A90093F82F3013F0010F25D040F2EC03C2F27C
S113A91000031B7813F0010F40F2F803C2F20003A6
S113A9201FBF07225A7600229A7612BF1A82062285
S113A9305A76012049F6D523C0F20003984740F225
S113A940EC03C2F2000310221A7048F2C933C0F2B9
S113A950000398475FE040F2EC03C2F200031B7867
S113A96013F0010F08D040F2F803C2F200030522ED
S113A9705A7600221A82E2E040F2E003C2F20003B7
S113A9801B88002B47D1DAE040F2E003C2F2000357
S113A990188820B149F6D523C0F20003984740F245
S113A9A02813C2F2000393F82F3013F0010F19D0CB
S113A9B040F2F803C2F2000307225A7600229A7684
S113A9C0012049F6D523C0F20003984740F2EC0376
S113A9D0C2F2000310221A7048F2C933C0F2000315
S113A9E0984718E040F2E003C2F200031B8893B9D1
S113A9F0A5E040F2EC03C2F200031B7813F0010F50
S113AA0000F09D8040F2F803C2F2000307225A7658
S113AA1000229A7693E040F22813C2F20003102237
S113AA2083F82F2040F2F804C2F2000440F2E0035D
S113AA30C2F2000328221A8040F22813C2F2000353
S113AA40502283F82E20227A40F22813C2F2000307
S113AA5083F82A20627A83F82B20A27A83F82C20A8
S113AA60E27A83F82D20227B83F82620627B83F808
S113AA702720A27B83F82820E27B83F82920062262
S113AA80DA75A2885A84E2889A8440F22412C2F2C7
S113AA9000021188598352889A832288DA83628853
S113AAA01A84637E13F0100F40F22813C2F20003DD
S113AAB01DBF002283F8312083F83020062202BF14
S113AAC083F830200A2283F8312040F22814C2F29D
S113AAD000044023A37540F2E003C2F200031B8884
S113AAE01A0A22746374002584F8355084F83450AB
S113AAF0658649F63933C0F200039847C04360863F
S113AB004523A373E5736575257540F26203C2F2AC
S113AB1000031A88013292B21A80130AA374E274F1
S113AB20258349F60D33C0F200039847C0432083C0
S113AB3040F2EC03C2F2000300221A7038BD40F266
S113AB40E003C2F2000300221A8040F2EC03C2F2D6
S113AB5000031A7038BD40F27403C2F200030121ED
S113AB601970FFF776BA40F27403C2F200030122AF
S113AB701A70E4E7030A43EA002080B2704700BF7A
S113AB802DE9F00340F27603C2F200034FF0000C0B
S113AB9083F800C040F27805C2F200052B4601227A
S113ABA01F461C88CCB15E88BEB1B0F80080A045B9
S113ABB013D14488B44210D140F27603C2F20003A8
S113ABC083F800C0086878608B883B8140F2D90321
S113ABD0C2F200031B78BB725AE0541CE4B20C337B
S113ABE0092C02D094462246DAE72B4600221E4660
S113ABF01C884CB95C883CB940F27603C2F200036D
S113AC001A70082A36D104E00132D2B20C33082A71
S113AC10EDD1002340F2D902C2F200021678B04608
S113AC201F4699465FFA83FCAA7AC2EB0804BC4229
S113AC30C2BFC2EB0602E146D7B201330C35082B82
S113AC40F0D140F27703C2F200031F7040F2D80340
S113AC50C2F2000383F8009040F27603C2F20003CC
S113AC6083F8009040F27803C2F2000309EB49092B
S113AC7003EB89060268334643F8042B0A687260C2
S113AC808A889A8040F2D903C2F200031B78B37217
S113AC90BDE8F003704700BFF0B440F2D903C2F23C
S113ACA000031E780136F6B21E7040F27803C2F239
S113ACB000030122002740F27604C2F200045888FF
S113ACC01988014389B259B1997A711A772907DD34
S113ACD0194601F8017B5F70013101F8017B0F70A7
S113ACE022700132D2B20C33092AE8D1F0BC704789
S113ACF038B540F2E003C2F200031B88292B06D8C2
S113AD0040F2E003C2F2000300221A8038BD40F290
S113AD10E003C2F2000300221A8040F22813C2F2B8
S113AD2000039B8AB3F5807F03D0B3F5007F5CD02A
S113AD3038BD40F22812C2F2000240F22413C2F2DB
S113AD400003D28C1B889A426FD140F22812C2F2BF
S113AD50000240F22413C2F20003128D5B889A426F
S113AD6063D1324CA51F204629464AF68133C0F2EE
S113AD7000039847A4F11C03002204F8082C0222C3
S113AD8004F8072C54F8062C626034F8022C228153
S113AD9040F26C02C2F20002106844F8060C928879
S113ADA024F8022C44F8160C24F8122C626844F897
S113ADB01C2C228924F8182C9A8B62816288A28127
S113ADC040F22412C2F200021188998352886280F0
S113ADD0082204F8102C062204F80F2C40F2E00399
S113ADE0C2F200032A221A8038BD40F22812C2F2AD
S113ADF0000240F22413C2F20003D28C1B889A4250
S113AE0013D140F22812C2F2000240F22413C2F21B
S113AE100003128D5B889A4207D10449084606391B
S113AE204AF68133C0F20003984738BD440100203C
S113AE3038B540F22813C2F20003D98B8AB24FF618
S113AE40FF739A4215D140F22813C2F20003188C02
S113AE504FF6FF7398420CD140F22813C2F200035C
S113AE604BF2B012C0F200021068186092889A8007
S113AE70B0E040F22413C2F200031B885A4040F2AF
S113AE802013C2F200031B881A4212D140F2281385
S113AE90C2F200031A8C90B240F22413C2F20003EF
S113AEA05B88584040F22013C2F200035B881842CA
S113AEB00CD040F2DC03C2F2000340F21C12C2F2D6
S113AEC000021188198052885A8005E040F2DC03A0
S113AED0C2F2000319805A8040F2DC03C2F200037C
S113AEE018885D8840F27803C2F2000300221C46F1
S113AEF0198881420AD15988A94207D140F27603C0
S113AF00C2F200031A70082A5BD109E00132D2B2FE
S113AF100C33082AEBD140F27603C2F200031A7014
S113AF2040F22814C2F200042046FF2106224BF20C
S113AF300903C0F200039847002384F8203084F802
S113AF40213084F8223084F8233084F8243084F8C3
S113AF50253040F26C02C2F200021168C4F80610F7
S113AF6092886281C4F81610628340F2DC02C2F255
S113AF7000021188E1845288228540F22412C2F230
S113AF8000021188A1835288E2832375012262752D
S113AF90A373E2730822227463740623A374042344
S113AFA0E37422730623637340F2F003C2F20003D6
S113AFB036341C6040F2E003C2F200032A221A80F5
S113AFC038BD40F22813C2F2000354F8040F18608D
S113AFD0A2889A8040F22813C2F2000340F26C0265
S113AFE0C2F200021168C3F8061092885A8108223E
S113AFF01A7300225A7340F2E003C2F200031A8863
S113B0000E321A8038BD00BF8307F0B448D0541EF6
S113B010002A43D0CDB2034602E0002C3ED01446B1
S113B02003F8015B13F0030F04F1FF32F5D1032C95
S113B0302DD9CDB20F2C45EA052545EA054518D989
S113B040A4F1100703F110061A463F0906EB071690
S113B0501560103242F80C5C42F8085C42F8045C5B
S113B060B242F5D104F00F040137032C03EB0713AC
S113B0700DD91E462246043A46F8045B032AFAD840
S113B080221F04F0030422F00302043213442CB1FF
S113B090C9B21C4403F8011BA342FBD1F0BC7047A6
S113B0A014460346C3E700BF6C69622F6472697675
S113B0B065726C69622F65746865726E65742E635F
S113B0C0000000006C69622F6472697665726C69B5
S113B0D0622F666C6173682E630000006C69622FD6
S113B0E06472697665726C69622F6770696F2E632A
S113B0F00000000040420F0000201C0080841E005D
S113B10000802500999E36000040380000093D006B
S113B11000803E0000004B00404B4C0000204E00DD
S113B120808D5B0000C05D000080700000127A001A
S113B13000007D0080969800001BB7000080BB00D3
S113B140C0E8CE00647ADA000024F4000000FA00BB
S113B1506C69622F6472697665726C69622F7379A7
S113B1607363746C2E63000000E10F4004E10F4030
S113B17008E10F4040E00F4044E00F4048E00F403A
S113B1806C69622F6472697665726C69622F737977
S113B190737469636B2E63006C69622F64726976E1
S113B1A065726C69622F756172742E630000000011
S10BB1B0FFFFFFFFFFFF000099
S90380007C
